:020000020000FC
:0200000019C025
:02000C00F0C141
:100034000FE50DBF04E00EBF55D416D301E01CD369
:10004400B3D3DED3E3D304E0E7D340E030E1B4D567
:1000540045E003E00BBD0FE10ABD0AE00EBD00E080
:100064000FBD00E109BF00E0009374000093760027
:10007400009377000093780000937500502F7894D4
:100084008D9A9598C4E0D0E000EF00937B0031FF97
:1000940001C0E1D45F9952D137FD06D005B70F7086
:1000A400006805BF8895F3CFEF93FF9334FF38C002
:1000B40083D5413059F400E010E09ED40F9306E05C
:1000C40011E0B1D30F91D9D3BAD329C0423059F436
:1000D40001E010E091D40F9306E011E0A4D30F9156
:1000E400CCD3ADD31CC0443011F482D518C04930F0
:1000F40031F406E011E097D3A9D5BFD3A0D34A3099
:1001040071F410E002E078D4009381009FD500934D
:100114007C0001E000937D0000E000937E000AC1B2
:10012400413019F500E010E067D40F9306E011E0C8
:100134007AD30F91A2D383D333FF05C0039504363A
:1001440040F000E006C032FF0FC00A9500300AF408
:1001540003E610E020E059D40F9306E011E063D3E6
:100164000F918BD36CD35BD4E5C0423019F501E019
:1001740010E042D40F9306E011E055D30F917DD3E4
:100184005ED333FF05C00395043640F000E006C09B
:1001940032FF0FC00A9500300AF403E611E020E0B4
:1001A40034D40F9306E011E03ED30F9166D347D3C6
:1001B40036D4C0C0433069F433FF0AC030D40AE0F7
:1001C40010E031D33090790040907A00552483D3E5
:1001D400B1C0443091F400917B0033FF05C0039516
:1001E400013F38F001E005C032FF06C00A9509F46A
:1001F40000EF00937B00FCD49DC0453051F433FFE5
:1002040007C0C8D4EEECFEE0059115910CD320D3C1
:1002140091C04630B1F433FF0AC0A1E0B0E03160D0
:10022400EAEAFEE005911591FED212D309C032FF2D
:1002340007C03E7FE2EBFEE005911591F4D208D3AE
:1002440079C0473081F433FF0DC0EAEBFEE005913D
:100254001591E9D2FDD227D4E4ECFEE00591159185
:10026400E2D2F6D267C0483051F433FF07C0D6D487
:10027400ECEDFEE005911591D6D2EAD25BC049308F
:10028400F1F406E011E0CFD2E1D4F7D2D8D233FFB3
:1002940005C00395053040F001E006C032FF0EC0F2
:1002A4000A9501300AF404E014EE21E0AED30F9372
:1002B40006E011E0B8D20F91E0D2C1D23BC04A307F
:1002C400C9F533FF0BC000917E0010917C00010F33
:1002D400109181001395011768F02BC032FF29C0DB
:1002E40000917E0010917C00011B011B08F400E0CA
:1002F40000937E0007E010E096D200917E00BDD20C
:100304009ED20BE010E0ACD400917C00023088F067
:1003140000E011E0A5D400917C00033050F005E02A
:1003240011E09ED400917C00043018F00AE011E042
:1003340097D400C03376FF91EF910895EAD2053641
:1003440011F46DD34DC0083611F460D249C00336A0
:1003540011F456D245C0093611F426D241C00337F0
:1003640039F402D310E020E050D30AE0A6D438C018
:100374000D3639F4F9D211E020E047D30AE09DD4D8
:100384002FC0073621F4A1E0B0E0316029C0023665
:1003940011F43E7F25C0013659F40AE08ED410E0F2
:1003A40002E02AD374D2C4D2052F71D2C1D218C0AC
:1003B400043711F478D314C00F3611F4CED310C01F
:1003C4000C3611F4E7D30CC00F3411F4D6D308C0A3
:1003D4000B3611F4A9D304C00B3411F4D5D300C0E7
:1003E4000AE08FD20DE08DD208950F930FB70F93CB
:1003F4001F930091740003950931C9F100937400AF
:10040400009174000130C9F4849905C06395653086
:1004140008F064E001C06627839905C073957530C0
:1004240008F070E001C07727829905C08395853074
:1004340008F080E001C0882763C000917400023096
:10044400A9F4633039F43F7E43954B3008F041E022
:1004540030690BC0733021F434FD07C0386805C01F
:10046400833021F434FD01C034684AC049C00027F8
:1004740000937400009175000395023361F00093BA
:10048400750030FF06C000917500013310F0959A95
:1004940037C0959835C000270093750030FF0FC012
:1004A400119709F00CC0326010917B00511710F0C5
:1004B4003E7F05C0A0917900B0917A0053950091D8
:1004C400760003950C3319F00093760019C00027C9
:1004D400009376000091770003950C3319F0009394
:1004E40077000EC0002700937700009178000395F1
:1004F400083119F00093780003C0002700937800B6
:100504001F910F910FBF0F91189507D0632C742C76
:10051400852C03D002D005D00895330C441C551CFF
:100524000895360C471C581C089536184708580877
:1005340008950F931F9310E0300E411E511E1F911A
:100544000F9108959F92AF92BF92212E962CA72CC3
:10055400B82C662477248824330C441C551C661C50
:10056400771C881C69147A048B0420F069187A08B3
:100574008B0833942A9481F7BF90AF909F9008958D
:100584001A3340F01F7D173408F009C0113438F0D5
:10059400175303C0103318F01F70889408950894FB
:1005A40008950F700A300CF0095F005D08952F93D1
:1005B4002FB70F93F6DF102F0F910295F2DF2FBFA5
:1005C4002F9108950F932F932227E0E6F0E00AE09D
:1005D400602E7724882418E1B5DF062D006301938B
:1005E40023950AE0602E772488243614470458049F
:1005F40094F7032D00630193239500E00083122FE9
:100604002F910F9108956F921F931FB70F9300E1DD
:10061400602E0F9155244424262E372E3694279489
:1006240010F4480E591E57944794379427946A94AB
:10063400B9F71FBF1F916F9008950F931F931FB7B2
:100644005694479437942794569447943794279410
:1006540000E8201628F001E0300E00E0401E501E95
:100664001FBF1F910F9108950F9300E407B905E888
:1006740006B9479A0F9108950F931F932F933F93B1
:100684004F9333244424552441E0202F302F222338
:1006940019F0440F2A95FCCF369A3699FECF04B14F
:1006A40015B1300E411E521E4A95B1F7332331F075
:1006B40056944794379427953A95C9F7203818F0FB
:1006C400339409F443944F913F912F911F910F91CB
:1006D40008951F931FB71F9317B1107F0770102B36
:1006E40017B91F911FBF1F9108950F931F932F9345
:1006F4002FB72F93102F02950F70969A28B3207F4F
:10070400022B08BB2AD0969A1F7028B3207F122B85
:1007140018BB23D028D02F912FBF2F911F910F9159
:1007240008950F931F932F932FB72F93102F029594
:100734000F70969828B3207F022B08BB0ED0969892
:100744001F7028B3207F122B18BB07D00CD02F9119
:100754002FBF2F911F910F910895979A00000000C9
:100764000000979808950F930FB70F9300E50000CA
:1007740000000A95E1F70F910FBF0F9108950F93B1
:100784000FB70F931F9302E405C00F930FB70F9396
:100794001F9306E119EC1A95F1F70A95D9F71F9101
:1007A4000F910FBF0F9108950F931F931FB72F93AE
:1007B40007B30F6007BB8E9A8F9A26E09698979896
:1007C400DEDF2A95E9F703E028B3207F022B08BB7C
:1007D400C4DFD5DFC2DFD3DFC0DFD1DF02E028B35F
:1007E400207F022B08BBB9DFCADF0CE29ADF0FE0DF
:1007F40098DF04E096DF2F911FBF1F910F9108959A
:100804000F9301E08EDFC1DF0F9108950F9302E093
:1008140088DFBBDF0F9108950F930770086081DFB5
:10082400A2DF0F9108950F931F930F71117010FDA4
:1008340010E4012B006875DF1F910F9108950F9349
:100844000FB70F9300E251DF0F910FBF0F9108957F
:100854000F930FB70F930591003011F046DFFBCFD4
:100864000F910FBF0F9108950F931F93A0DE3DDFEB
:10087400012F3BDF1F910F9108950F931F932F9327
:100884002FB72F9317E7E12F13E0F12F09C00F9330
:100894001F932F932FB72F9313E8E12F14E0F12F19
:1008A400102F00E3145610F00395FCCF202F0033D3
:1008B40009F009951C5900E31A5010F00395FCCF78
:1008C4000995165F00E3010F09952F912FBF2F9112
:1008D4001F910F91089518E175DE029106DF1A95B4
:1008E400E1F708950F9300E000BD03E309B906E8BA
:1008F40000BD539A549A0F91089505E502D0FDCF97
:1009040008955D9BFECF0CB908955F9BFECF0CB19B
:1009140008955F9BFECF0CB1F4DF08950F930AE0B6
:10092400F0DF0F9108950F930DE0EBDF0F91089521
:100934000F930AE0E6DFF8CF0F930CE0E2DF0F91AC
:1009440008951F932F93E1DF102F1ADEE0F3D9DF10
:10095400212F2295DADF102F13DEE0F3D2DF012FEF
:10096400022B2F911F910895D0DF0F70000F102ECE
:10097400110C110C100EC9DF0F70010D08950F93A7
:100984001F9315DEBEDF012FBCDF1F910F91089569
:100994000F930591003011F0B4DFFBCF0F91089550
:1009A4000F931F931FB7E0E6F0E02224B2DF0D306F
:1009B40021F00F7001932394F9CF5F99A6DF3324BC
:1009C40044245524E0E6F0E00191B3DD2A9411F0CB
:1009D4009CDDFACF1FBF1F910F9108950F931F93B2
:1009E400EF93FF93EFDD02918CDF1A95E1F7FF910E
:1009F400EF911F910F910895E199FECFF8940EBBEA
:100A04001FBBE09A0DB378940895E199FECFF89452
:100A14001EBB2FBB0DBBE29AE19A789408950AE0BD
:100A24004CD110E001E0E8DF7727602F99278CE3B1
:100A3400EADD10E000E0E0DF1127200E311E2092F5
:100A4400790030927A00A22DB32D37FD03C0432CD8
:100A5400322CC4DF0895FF92F9D0902FFF240F2D7C
:100A640038DE03E009DE032D1C2F2D2FCEDF219667
:100A7400042D1C2F2D2FC9DF2196052F00938100F3
:100A840012E020E0C2DFF3949A9549F73D7F00E03D
:100A940011E0C9DE052FF1DE00E227DE1CDF00E2F3
:100AA40024DEFF900895CF93DF935F930FB70F93E6
:100AB4000AE003D110E002E09FDF502FE8DE38DFC8
:100AC4005EDE552359F111E004EE96DFE0DE30DFFF
:100AD40056DE10E001E090DF7727602F99278CE342
:100AE40092DD10E000E088DF1127200E311E432C38
:100AF400322C74DF1DDF43DEC4E0D0E055240C2F1C
:100B04001D2F7ADF302E21960C2F1D2F75DF402EDE
:100B1400219664DF0DDF33DE5A9589F70F910FBFFD
:100B24005F91DF91CF9108951F932F932FB72F9348
:100B340037DF442079F4032D053060F4332011F4B9
:100B440001E0302E14EE21E060DF2F912FBF2F91B2
:100B54001F910895E4EEFCE0F8CF22DF442051F425
:100B6400032D013F38F4332011F401E0302E30928C
:100B74007B000895E4EEFCE0FCCF0AE09ED00091F7
:100B84007B0085DED5DE08950AE097D05FD07FDE56
:100B9400CFDE089509C01C2F2D2F0FEF36DF2196CD
:100BA40001E0C43ED007B8F300E0502F12E020E08B
:100BB4002CDFC4E0D0E008950F930FB70F931F9379
:100BC4002F931EDE042F25E01127000F111F2A95F5
:100BD400E1F7EAE4FDE0E00FF11F3ADE00E011E0A6
:100BE40022DE36DE2F911F910F910FBF0F910895D2
:100BF4000F931F931FB71F930DE010E014DE052F12
:100C04003CDE1DDE06E011E00EDE00917B0035DEE9
:100C140016DE1F911FBF1F910F9108950F931F930D
:100C24002F932FB72F9302E010E020E0EEDE00E0D8
:100C340011E020E0EADEF3DE01E014EE21E0E5DE7F
:100C44002F912FBF2F911F910F9108951F932F93D1
:100C54002FB704EE11E0D0DE2FBF2F911F9108951E
:100C6400EF93EFB7EF93FF933F924F925F92DBDDE9
:100C7400E4E0F0E000917E0010E0512E000F111F1F
:100C8400E00FF11F0E2F1F2FB7DE302E31960E2FDF
:100C94001F2FB2DE402E00917E00039500937E004C
:100CA4001ADECDDD5F904F903F90FF91EF91EFBF43
:100CB400EF910895ECDD00E224CE1F931FB75FDDB2
:100CC4000A95E9F71FBF1F9108952077757264652F
:100CD4002065696E67657374656C6C742E20000002
:100CE4000A0D204620452048204C20452052202132
:100CF400212120576572742067726F657373657262
:100D04002032343020212100084269747465206542
:100D1400696E65205A61686C2067726F65737365CC
:100D24007220302061626572206B6C65696E657239
:100D3400203234302065696E676562656E3A200042
:100D4400546573742000446174656E6C6F676765E5
:100D540072204D3820004D454E55455741484C2092
:100D64002D3E2054310050415553452053454B5599
:100D74004E44454E3A002020765433205F5F5F2076
:100D840054325E2020005041555345204D494E5564
:100D940054454E3A20002020765433205F5F5F2074
:100DA40054325E202000494E54455256414C4C204A
:100DB4005F5F5F2073002020205432203D20474F86
:100DC4002020202020005745525445204D415820D2
:100DD400414B545F5F002020765433205F5F5F20D7
:100DE40054325E2020005745525445204C4F455301
:100DF4004348454E20002020205432203D20474FB8
:100E04002020202020004D45535352454948452079
:100E140020202020200054323D474F202054333DD1
:100E240053544F50500057455254452053454E4457
:100E3400454E202020005432203D20474F202020C2
:100E440020202020200044454641554C545A454911
:100E5400542F4B414E002020205432203D20474F38
:100E64002020202020004D4553534B414E41454CFA
:100E7400453A202020002020765433205F5F5F20F5
:100E840054325E20200057455254453A205F5F5F3C
:100E9400205F5F5F5F005F5F5F5F205F5F5F5F207A
:100EA4005F5F5F5F20000A002D414E2D20000A0085
:100EB4002D4155532D00080153454E44494E4700DA
:100EC4000801202020202020200003012047454C39
:100ED4004F455343485420000301202047455345C0
:060EE400545A54202000C6
:00000001FF
